:100000003EC1000058C1000056C1000054C10000AC
:1000100052C1000050C100004EC100004CC10000A0
:100020004AC1000048C1000046C100000C94C70B43
:1000300042C1000040C100003EC100003CC10000C0
:100040003AC1000038C1000036C1000034C10000D0
:1000500032C1000030C100002EC100002CC10000E0
:100060002AC1000028C1000026C1000024C10000F0
:1000700022C10000A602AB02B602C002C602CC0238
:10008000F802040309030E031D0322032D034C038E
:10009000600366036E0374037A038203D303EF03E2
:1000A00000040B0410050C051405180512050E05B7
:1000B00016051A05920CB20C980DB20C980DF40CA2
:1000C000160D980D690D7B0D2203690062006D000D
:1000D0002D00630061007000730065006E00730006
:1000E00065002D00750073006200000022035400BB
:1000F0006F006D00200057006F006E0067002D003C
:1001000043006F0072006E0061006C006C00000024
:10011000040309040902540003010080FA090400E1
:10012000000103010100092111010001222500073E
:1001300005810308000A0904010001030000000909
:1001400021110100012220000705830308000A098C
:10015000040200010300000009211101000122BE78
:10016000000705820319000A120110010000002097
:10017000810402000100010200010600FF0901A143
:10018000010902150025FF7508950881020903156C
:100190000025FF750895089102C005010906A10117
:1001A0000508190129031500250195037501910220
:1001B000950175059101050719E029E7150025014D
:1001C00095087501810205071900293115002501DF
:1001D0009532750181029501750181010507193379
:1001E000299B15002501956975018102950175010D
:1001F00081010507199D29A41500250195087501A0
:1002000081020501198129831500250195037501D6
:100210008102050C19B029B8150025019509750151
:100220008102050C09CD09E209E909EA0A8A010AF5
:1002300092010A94010A21020A23020A24020A25D1
:10024000020A27020A2A0215002501950D7501816F
:1002500002950175028101C005010906A101750120
:100260009508810195017508810195057501910138
:10027000950175039101950675088101C00011244F
:100280001FBECFEFD4E0DEBFCDBF11E0A0E0B1E0F4
:10029000EAE7F0E202C005900D92A635B107D9F762
:1002A00013E0A6E5B1E001C01D92A837B107E1F760
:1002B0008CD00C943B10A4CE80E291E00E94FD0E05
:1002C00080E191E00E94FD0E80E091E00E94FD0E31
:1002D000E2EEF0E0808184608083B2C280E291E04F
:1002E0000E94CD0D80E191E00E94CD0D80E091E073
:1002F0000C94CD0D80912E0190912F01009729F043
:10030000019790932F0180932E0180911E0190916F
:100310001F01009729F0019790931F0180931E0100
:1003200080910E0190910F01009729F00197909311
:100330000F0180930E0192C20F931F93CF93DF930F
:10034000FC01C901E80121E0E032F20711F4FBD21F
:1003500005C021E0E031F20721F484D188E090E08B
:1003600005C06681778181D389E190E09983888394
:1003700080E0DF91CF911F910F910895AC01C901E9
:1003800021E04032520709F44AC44051514009F477
:10039000D1C048C484B7877F84BF88E10FB6F89482
:1003A00080936000109260000FBE90E080E80FB66E
:1003B000F89480936100909361000FBEE1D612D74C
:1003C0003AD214D7469A0C94B80BE4DF7894ACD2A6
:1003D000BAD543D691D28FE19EE40197F1F700C0E0
:1003E0000000EED680916A0390916B03019609F4A8
:1003F000DAD41BD480E291E00E94100F80E191E0FA
:100400000E94100F80E091E00E94100F0E94B10D39
:10041000F0CF292F332723303105A9F06CF4213098
:10042000310509F442C02230310509F043C084E5AA
:1004300090E024E131E042C021323105C9F022329E
:10044000310519F137C099278130910541F082308B
:10045000910541F0892B71F5E0E1F1E005C0ECEE8A
:10046000F0E002C0E8ECF0E0849190E09F0126C04B
:10047000633000F5E62FF0E0EE0FFF1FE25CFE4F69
:100480002081318189E090E019C0633098F4E62F33
:10049000F0E0DF01AA0FBB1FA85CBE4F2D913C917D
:1004A000EB5CFE4F808190E009C082E190E028E69D
:1004B00031E004C080E090E020E030E0FA013183D8
:1004C00020830895EF92FF920F931F93CF93DF93B2
:1004D00051E0EE24E394F12C461728F1E62FF0E0EA
:1004E000EE0FFF1FEE0FFF1FE957FE4F20E030E039
:1004F000DC01A50FB11D8F01020F131FE8017881E8
:1005000073304CF07C918701022E01C0000F0A94D9
:10051000EAF7702B7C932F5F3F4F2430310559F75A
:100520006F5F5F5FD9CFDF91CF911F910F91FF90E8
:10053000EF900895DC014C9150E04D30510508F0EA
:1005400090C0465C5F4FFA010C94DF0F11968C91BE
:1005500080933201089511962C91119712968C91E7
:1005600090E0982F8827820F911D0BC611968C91D1
:10057000882309F476C0E0913301F09134010994A5
:1005800011968C91882309F46CC010C611968C9139
:10059000882309F466C007C413963C9113971296FA
:1005A0002C9112971196AC91EA2FEF73E73108F076
:1005B00058C0243008F055C0A295A695A695A37002
:1005C000A150A33040F4B0E0AA0FBB1FAC5BBE4FFC
:1005D0008D919C9102C08EE492E0F0E0EE0FFF1F3F
:1005E000EE0FFF1FE20FF11DE80FF91F3083089592
:1005F00012968C9112971196EC91E83090F5F0E0FC
:10060000EA5FFC4F8083089511968C91882349F10D
:1006100024C511968C91882321F13AC513968C91AB
:10062000139712969C91129711962C912093850105
:10063000909384018093860103C111968C91882345
:1006400081F048C111968D919D91AC918093E30109
:100650009093E401A093E501089511968C91811186
:100660006AC408950F931F93CF93DF938C0188E0A2
:10067000D8011D928A95E9F740913201F801408333
:1006800050E0415051094B30510508F0CFC0495B53
:100690005F4FFA010C94DF0F84E0D80111968C9320
:1006A000119798E012969C93129797E113969C935A
:1006B000139714968C93149781E015968C93B6C07B
:1006C00046E060E0C801FEDE83E005C04DE067E083
:1006D000C801F8DE84E080933201A8C044E16EE0F6
:1006E000C801F0DE85E0F7CF47E165E1C801EADE49
:1006F00082E0F1CF90916A0380916B03F8019183BE
:10070000828394C05091810140918001852F829510
:10071000880F880F807C842BD80111968C93F80168
:100720003296842F90E0880F991F880F991F20918F
:10073000300130913101280F391F80E090E0D9015C
:10074000A80FB91F6C916193019684309105B9F798
:100750004F5F40938001473109F068C010928001DB
:1007600081E0850F843019F08093810102C01092DE
:10077000810180918101813061F040F0823061F02F
:10078000833009F053C08AEA92E008C08EE492E018
:1007900005C08EE093E002C082EF91E090933101BA
:1007A0008093300143C080917F01F8018183A82F9D
:1007B000B0E0AA0FBB1FAA0FBB1FAA5FBC4F4D9191
:1007C0005D916D917C9142835383648375838F5FC8
:1007D00080937F01823051F510927F0127C0A0E500
:1007E000B1E0E801219681E08F5F9D919993992373
:1007F00011F08730C9F7F801E80FF11D108216C01B
:1008000080918501F80181838091840182838091A8
:10081000860183830BC02091E3013091E401409174
:10082000E501D80111962D933D934C93DF91CF9123
:100830001F910F910895249A259A269A279A089530
:10084000109283012C982D982E982F9880918501D5
:10085000813019F42F9A10928201089580918301BA
:100860008F3F19F08F5F80938301809185018130E4
:10087000B1F49091830180918401981302C02E9865
:10088000089580918201882351F02091860192176A
:1008900030F0109283018150809382012E9A089546
:1008A000809182018F5F80938201089590918501EC
:1008B000923079F480FF02C02D9A01C02D9881FFFB
:1008C00002C02E9A01C02E9882FF02C02C9A089571
:1008D0002C980895609185018AE791E00E94291083
:1008E000609184018BE791E00E942910609186015C
:1008F0008CE791E00C9429108AE791E00E94121095
:10090000833018F48093850102C0109285018BE733
:1009100091E00E941210809384018CE791E00E9484
:1009200012108093860108958CE5E7E8F1E0DF017D
:100930001D928A95E9F78CE0E6EEF1E0DF011D9269
:100940008A95E9F708958F929F92AF92BF92DF92B6
:10095000EF92FF920F931F93CF93DF93EC01B3D3EA
:100960008150833048F4E82FF0E0EE0FFF1FE65B84
:10097000FE4FA081B18102C0AEE4B2E020E030E0E1
:10098000F12C01E010E0490195948794DF2C80E080
:1009900090E0A4014A515E4F4A01522F5170E52E5A
:1009A000F5E0FF1508F44EC0F401608170E0EE2020
:1009B00059F0AC014C5F5F4F580102C0AA0CBB1C40
:1009C0004A95E2F7A50107C0A801082E02C0440F0E
:1009D000551F0A94E2F746235723452B69F1AD01D1
:1009E000480F591FFA014081443030F150E3540F51
:1009F000533010F1F394BE016D0D711DFB01428364
:100A000050E0405E510948305105B0F44E5A5F4FF6
:100A10006881FA010C94DF0F6E5F0DC0605E0BC041
:100A20006F5F09C0605F07C06C5F05C0605C03C09A
:100A3000685F01C06058688301968430910511F0A9
:100A4000DF2CAECF2F5F3F4F14962731310509F0D1
:100A50009ACFDF91CF911F910F91FF90EF90DF9090
:100A6000BF90AF909F908F9008952F923F924F929A
:100A70005F926F927F928F929F92AF92BF92CF922E
:100A8000DF92EF92FF920F931F93CF93DF9300D0EB
:100A90001F92CDB7DEB79B838A835B0114D381504D
:100AA000833048F4E82FF0E0EE0FFF1FE65BFE4FC7
:100AB0008081918102C08EE492E03C01E12CF12C16
:100AC00088248394912C6701D594C79400E010E0AA
:100AD000C6018A519E4F6C019E2D9170392EF601F0
:100AE000208130E0332051F0C8010496A40102C0F7
:100AF000440F551F8A95E2F7CA0107C0C401002EB2
:100B000002C0880F991F0A94E2F782239323892B4E
:100B100009F456C0F301E00FF11F2081213E99F046
:100B200060F4233D38F4203D08F04AC0233008F437
:100B300047C025C0203EB1F022C0253E21F090F0F4
:100B4000283EE8F40FC0F501808190E030E2320FDA
:100B500002C0959587953A95E2F780FD03C02983F9
:100B60009FDE2981205EC401022E01C0880F0A94F5
:100B7000EAF7EA81FB819081982B908321C0422E75
:100B8000469446944694512C2770222EF501E40D8C
:100B9000F51D818190E0022E02C0959587950A94FB
:100BA000E2F780FF7DDEEA81FB81E40DF51DC401E3
:100BB000022C01C0880F0A94EAF79181982B918347
:100BC0000F5F1F4F0430110509F089CFFFEFEF1AB7
:100BD000FF0A44E0640E711C57E1E516F10409F0C8
:100BE00072CFEA81FB818181887F8183838D887FB9
:100BF000838F0F900F900F90DF91CF911F910F91E6
:100C0000FF90EF90DF90CF90BF90AF909F908F902C
:100C10007F906F905F904F903F902F900895FC01D0
:100C2000808144CEFC01808141CE4F925F926F92D1
:100C30007F928F929F92AF92BF92CF92DF92EF926C
:100C4000FF920F931F93CF93DF9300D000D0CDB7C7
:100C5000DEB78CE0E6EEF1E0DF011D928A95E9F760
:100C600067E8E62E61E0F62E00E010E09924939408
:100C700075E0A72EDD24D394E8ECBE2EC02EE02F25
:100C8000E695E695E695F0E0ED51FE4F808190E027
:100C9000202F277002C0959587952A95E2F780FD51
:100CA00064C04698802FAAD2469A19821A821B8263
:100CB0001C82892D8A95F1F71899998219999A823F
:100CC0001A999B821B999C82980135952795AE01B4
:100CD0004F5F5F4F2701D70180E090E02A513E4FE0
:100CE000EC2DE1707E2E682EFA016191AF01F201C8
:100CF000662319F06081615002C060816F5F60837C
:100D0000BD018C9087FE02C01C9204C0F5E0F8156E
:100D10000CF4AC921196FB0160816330B4F0F901E0
:100D20008080772051F0BC016C5F7F4FFD2D01C0AA
:100D3000FF0F6A95EAF76F2F05C06D2D01C0660F92
:100D40006A94EAF76829F90160830196FFEF4F1A68
:100D50005F0A8430910539F6469848D2469A66E192
:100D6000C61619F08B2D8A95F1F70F5F1F4F84E09F
:100D7000E80EF11C0731110509F080CF0F900F909C
:100D80000F900F90DF91CF911F910F91FF90EF90F7
:100D9000DF90CF90BF90AF909F908F907F906F909B
:100DA0005F904F900895AF92BF92CF92DF92EF92F3
:100DB000FF920F931F93CF93DF932EE432E0F12C39
:100DC000B12C80E090E0F901E80FF91F408141303B
:100DD00021F0423019F4B39401C0F39401968430A9
:100DE000910589F72C5F3F4F82E02A3A380749F78F
:100DF000C0E0D0E0CC24CA942FE0D22E00E010E076
:100E0000C601801B910B82309105C0F1EC01D69593
:100E1000C795C00FD11FCE01B4D18FE891E00197E3
:100E2000F1F700C0000090E2E92EFFDEEA94E9F756
:100E300027E831E04EE452E060E080E090E0F90124
:100E4000E80FF91F708173303CF0FA01E80FF91FC9
:100E50007081743008F06F5F01968430910579F7E6
:100E60002C5F3F4F4C5F5F4F91E0233E390729F7DE
:100E70006B1510F48E01C4CF6E01C2CF6E010FEF5F
:100E80001FE0A12CB12CC8018A199B098230910561
:100E9000C0F1EC01D695C795CA0DDB1DCE0171D10D
:100EA0008FE891E00197F1F700C00000B0E2EB2E6F
:100EB000BCDEEA94E9F747E851E08EE492E060E0B6
:100EC00020E030E0FA01E20FF31F708173303CF054
:100ED000FC01E20FF31F7081713009F46F5F2F5F27
:100EE0003F4F2430310571F74C5F5F4F049621E08E
:100EF000433E520729F76F1510F45E01C4CF8E01EF
:100F0000C2CFC6018C1B9D0BF4E096958795FA9590
:100F1000E1F76FE070E00E94CE0F8C0F9D1F31D182
:100F2000DF91CF911F910F91FF90EF90DF90CF90C5
:100F3000BF90AF9085CC43E050E06DE771E083EE69
:100F400091E00C941A1043E050E06DE771E083EEFD
:100F500091E00E9402108091E3018F3F71F4809133
:100F6000E4018F3F51F48091E5018F3F31F41092FD
:100F7000E3011092E4011092E50108958F929F928F
:100F8000AF92BF92CF92DF92EF92FF920F931F9397
:100F9000CF93DF936C014B01C0E0D0E07401EC0E05
:100FA000FD1E00E010E05601AC0EBD1EC8018A0D0A
:100FB0009B1D0E9412108F3F09F480E0F70181937E
:100FC0007F010F5F1F4F0430110581F72496CC3548
:100FD000D10521F7DF91CF911F910F91FF90EF90F5
:100FE000DF90CF90BF90AF909F908F9008958F9299
:100FF0009F92AF92BF92CF92DF92EF92FF920F93A8
:101000001F93CF93DF936C014B01C0E0D0E07401DC
:10101000EC0EFD1E00E010E05601AC0EBD1EF70107
:1010200061917F01C8018A0D9B1D0E9429100F5FED
:101030001F4F0430110599F72496CC35D10539F7A7
:10104000DF91CF911F910F91FF90EF90DF90CF90A4
:10105000BF90AF909F908F90089548E050E062E776
:1010600071E086E093E0CED76EE472E082E090E03B
:1010700085DF6EE073E08EE590E080DF62EF71E087
:101080008AEB90E07BDF6AEA72E086E191E076CF5E
:1010900048E050E062E771E086E093E0CBD76EE491
:1010A00072E082E090E0A3DF6EE073E08EE590E016
:1010B0009EDF62EF71E08AEB90E099DF6AEA72E00E
:1010C00086E191E094CF0F931F93CF93DF934EE48B
:1010D00052E020E030E0C0E061E070E0F901F59519
:1010E000E795EA51FE4FA081B0E080E090E0D22F7A
:1010F000D170DD2351F0FC0134968B0102C0000F4A
:10110000111FEA95E2F7F80107C0FB01082E02C0A3
:10111000EE0FFF1F0A94E2F7EA23FB23EF2B79F08F
:10112000FA01E80FF91FE081E13D31F0E23D31F0D5
:10113000E03D29F4C16003C0C26001C0C4600196F3
:1011400084309105B1F62F5F3F4F4C5F5F4F2731E1
:10115000310521F6CC2371F0E6E0F3E08191982F80
:1011600092959F709C1302C08F7005C013E0EE3003
:10117000F107A1F780E0DF91CF911F910F910895C2
:101180005BC0CF93DF9300D0CDB7DEB780936A0307
:1011900090936B039F7099838A8362E0CE010196DE
:1011A0007FD00F900F90DF91CF91089560916A03E7
:1011B00080E090E04ED760916B0381E090E049C7FA
:1011C000CF93DF9381E090E02DD7C82FD0E0DC2FC4
:1011D000CC2780E090E026D79E01282BC901DF9123
:1011E000CF91CFCF3C9A3D9A3E9A08954598449826
:1011F00088E1459A45988150E1F7089545984498CB
:10120000449A459A4598449890E0981721F0459A59
:1012100045989F5FFACF0895882321F05098489B06
:10122000FECF0895509A58980895882311F0519848
:101230000895519A59980895509A519A81E0F5DF8E
:1012400081E0EACF80E0F1DF00C080E0E5DF00C0B0
:1012500081E00895489B03C0509A5898089550988B
:10126000489BFECF0895CF93DF93D82FC8E08D2FF2
:10127000881F8827881FD9DFEDDF00C0EBDFDD0F77
:1012800000C0C150A1F75198E5DF499905C000C0E1
:10129000E1DF519A00C0C1E08C2FDF91CF9108951A
:1012A000EF92FF920F931F93CF93DF93182FF92E96
:1012B000062FC8DF811102C080E017C080ECD3DFA9
:1012C0008823D1F3E12EC12FDF2D10E08C2F8E1952
:1012D000801728F48991C7DF182F8111F7CF81E09B
:1012E0009BDF000081E0A1DF812FDF91CF911F9173
:1012F0000F91FF90EF900895CF92DF92EF92FF92BF
:101300000F931F93CF93DF937C018B01EA01C9D127
:10131000811131C0209731F088819981081B190B08
:10132000E80EF91EC12CD12C0115110519F180917F
:10133000E80085FD14C08091E8008E778093E80076
:1013400010D4209741F0888199818C0D9D1D99833F
:10135000888385E010C0A5D1882331F30CC0F70144
:1013600081917F018093F10001501109FFEFCF1AA5
:10137000DF0ADACF80E0DF91CF911F910F91FF90CC
:10138000EF90DF90CF90089520917603309177030E
:101390002617370748F06115710539F42091E800E8
:1013A0002E772093E80001C0B90120E06115710596
:1013B000D1F130916F03332309F441C0353009F482
:1013C00040C03091E80033FD38C03091E80032FF72
:1013D00006C08091E80082FF29C080E00895309126
:1013E000E80030FFE3CF2091F20030E0FC01281B41
:1013F000390BCF01820F931F6115710549F08032BF
:10140000910530F481918093F10061507109F1CF21
:1014100021E0809709F020E08091E8008E778093AA
:10142000E800CF01C3CF2111C4CFD3CF80916F0388
:10143000882329F0853069F604C081E0089582E0B0
:10144000089583E008956115710529F42091E8005D
:101450002B772093E8006115710521F120916F032E
:10146000222349F1253049F12091E80023FD1FC0D6
:101470002091E80022FFF2CFFC01CF012091F20081
:10148000222321F38091F1008193CF0161507109F2
:101490006115710591F7DACF80916F03882359F0B8
:1014A000853059F08091E80080FFF6CF02C081E0DE
:1014B000089580E0089582E0089583E008952091E2
:1014C0007603309177032617370748F061157105C9
:1014D00039F42091E8002E772093E80001C0B9018B
:1014E00020E061157105D9F130916F03332309F4C0
:1014F00042C0353009F441C03091E80033FD39C0B5
:101500003091E80032FF06C08091E80082FF2AC0D7
:1015100080E008953091E80030FFE3CF2091F200A1
:1015200030E0FC01281B390BC9018E0F9F1F61158C
:10153000710551F08032910538F484918093F10067
:10154000319661507109F0CF21E0809709F020E0D9
:101550008091E8008E778093E800CF01C2CF2111FF
:10156000C3CFD2CF80916F03882329F0853061F6F5
:1015700004C081E0089582E0089583E00895982FE3
:10158000953058F59093E900981739F07091EC0078
:101590002091ED005091F00003C0242F762F50E0F1
:1015A00021FF19C03091EB003E7F3093EB0030916A
:1015B000ED003D7F3093ED003091EB0031603093D2
:1015C000EB007093EC002093ED005093F00020911D
:1015D000EE0027FF07C09F5FD3CF8F708093E90095
:1015E00081E0089580E008950F931F93CF93DF93D8
:1015F000062FEC0110E0101769F19881992339F159
:101600002C81E981FA816B81892F8F70853010F0F0
:1016100080E021C0223010F056E001C052E028E006
:1016200030E040E02E173F0720F44F5F220F331FBA
:10163000F9CF4295407F452B991F9927991F6295B5
:10164000660F660F607C692B9ADF882309F31F5FA2
:101650002596D1CF81E0DF91CF911F910F91089511
:101660008091700387FD05C08091E80080FF0EC067
:1016700012C08091E80082FD05C080916F03811146
:10168000F8CF08958091E8008B7708C080916F03B0
:101690008111EACF08958091E8008E778093E80069
:1016A00008958091E4009091E50045E62091EC00DA
:1016B00020FF21C02091E80020FD21C020916F0370
:1016C000222389F0253089F02091EB0025FD0FC001
:1016D0002091E4003091E5002817390739F3415093
:1016E00041F0C901E3CF82E0089583E0089581E0ED
:1016F000089584E008952091E80022FFDFCF80E084
:1017000008953FD041D08091D8008F778093D80042
:101710008091D80080688093D8008091D8008F7D18
:101720008093D80084E089BD86E089BD09B400FEBD
:10173000FDCF10926F0310926C0310926D0342E282
:1017400060E080E01CDF8091E1008E7F8093E1000B
:101750008091E20081608093E2008091E2008860E5
:101760008093E2008091E0008E7F8093E0000895F6
:10177000E3E6F0E080818E7F808381E080936E03DA
:10178000C0CF1092E20008951092E10008951F92D8
:101790000F920FB60F9211242F933F934F935F93A5
:1017A0006F937F938F939F93AF93BF93EF93FF9329
:1017B0008091E10082FF0BC08091E20082FF07C0B0
:1017C0008091E1008B7F8093E1000E947A018091FB
:1017D000E10080FF17C08091E20080FF13C080917C
:1017E000E2008E7F8093E2008091E200806180932E
:1017F000E2008091D80080628093D80019BC1092DA
:101800006F03AED18091E10084FF2DC08091E20092
:1018100084FF29C084E089BD86E089BD09B400FE4B
:10182000FDCF8091D8008F7D8093D8008091E1001A
:101830008F7E8093E1008091E2008F7E8093E200B2
:101840008091E20081608093E20080916C038111BD
:1018500004C08091E30087FF02C084E001C081E002
:1018600080936F037DD18091E10083FF22C080913E
:10187000E20083FF1EC08091E100877F8093E1003A
:1018800082E080936F0310926C038091E1008E7F61
:101890008093E1008091E2008E7F8093E20080914E
:1018A000E20080618093E20042E260E080E067DE77
:1018B00057D1FF91EF91BF91AF919F918F917F9100
:1018C0006F915F914F913F912F910F900FBE0F90AD
:1018D0001F9018951F93CF93DF93CDB7DEB7AA97CC
:1018E0000FB6F894DEBF0FBECDBFE0E7F3E0809106
:1018F000F100819323E0E837F207C9F70E946E01F7
:101900008091E80083FF14C120917003309171032E
:10191000832F90E08A30910508F00AC1FC01E65A55
:10192000FF4F4DC3203881F0223809F001C180916A
:1019300074038F708093E9008091EB0085FB88270A
:1019400080F91092E90004C080916D03811182E05A
:101950009091E800977F9093E8008093F1001092B7
:10196000F100C2C0822F8D7F09F0E2C0222319F05E
:10197000223061F0DDC080917203813009F0D8C05F
:10198000333009F080E080936D0328C080917203AA
:10199000811124C0209174032F7009F4C9C02093D1
:1019A000E9008091EB0080FF19C08091EB0033309B
:1019B00011F4806211C080618093EB0081E090E0BF
:1019C000022E01C0880F0A94EAF78093EA00109271
:1019D000EA008091EB0088608093EB001092E900B0
:1019E0008091E800877F83C02111A2C0109172030B
:1019F0001F778091E3008078812B8093E3008091B2
:101A0000E800877F8093E8002BDE8091E80080FF6C
:101A1000FCCF8091E30080688093E300112311F0F4
:101A200083E001C082E080936F0382C0205822309F
:101A300008F07EC080917203909173038C3D23E087
:101A4000920771F583E08A838AE289834FB7F8941D
:101A5000DE01139620E03EE051E2E32FF0E05093E8
:101A60005700E49120FF03C0E295EF703F5FEF70F5
:101A70008E2F90E0EA3010F0C79601C0C0968D938B
:101A80009D932F5F243149F74FBF8091E800877FF6
:101A90008093E8006AE270E0CE01019675DC13C025
:101AA000AE014F5F5F4F609174030E94090200977F
:101AB00009F43EC02091E800277F2093E800BC0194
:101AC00089819A81FCDC8091E8008B778093E80023
:101AD0002FC0203869F58091E800877F8093E80067
:101AE00080916C038093F1008091E8008E77809361
:101AF000E800B6DD1DC021111BC090917203923029
:101B0000B8F48091E800877F8093E80090936C039D
:101B1000A7DD80916C03811104C08091E30087FFF1
:101B200002C084E001C081E080936F030E945C01E9
:101B30008091E80083FF0AC08091E800877F80934E
:101B4000E8008091EB0080628093EB00AA960FB6CC
:101B5000F894DEBF0FBECDBFDF91CF911F910895E6
:101B60000895CF9380916F038823A9F08091E900B5
:101B70008F709091EC0090FF02C090E801C090E05F
:101B8000C92FC82B1092E9008091E80083FDA2DEE6
:101B9000CF70C093E900CF9108956F927F928F929A
:101BA0009F92AF92BF92CF92DF92EF92FF920F93EC
:101BB0001F93CF93DF9300D01F92CDB7DEB77C0188
:101BC000ADB6BEB68091E80083FF00C1F701808109
:101BD00090E020917403309175032817390709F0BC
:101BE000F5C080917103833009F497C030F48130DF
:101BF00071F0823009F4CEC0E9C08A3009F4B2C075
:101C00008B3009F49BC0893009F0E0C048C0809156
:101C10007003813A09F0DAC08DB69EB61A82198235
:101C200080917203109173038B83F701408550E01C
:101C30008DB79EB7841B950B0FB6F8949EBF0FBE51
:101C40008DBFEDB7FEB731966F0160E070E0CF0158
:101C5000D2D14FEF410F8E010F5F1F4F9601BE0192
:101C60006D5F7F4FC7010E949C01F70186819781BC
:101C7000009721F0408550E0B601B4D11092E90000
:101C80008091E800877F8093E80069817A81C601AE
:101C90007BDB8091E8008B778093E80038C08091EF
:101CA0007003813209F092C08DB69EB60091760322
:101CB0001091770370907203609073038DB79EB795
:101CC000801B910B0FB6F8949EBF0FBE8DBFEDB772
:101CD000FEB731966F018091E800877F8093E8001E
:101CE000B801CF01B0DB8091E8008E778093E800E7
:101CF00021E0711001C020E030E0021B130B2C0D1D
:101D00003D1D4FEF460D672DC7010E94BE010FB666
:101D1000F8949EBE0FBE8DBE59C080917003813A6B
:101D200009F054C08091E800877F8093E80080919B
:101D3000E80080FFFCCFF701818540C080917003EF
:101D4000813209F043C08091E800877F8093E800EA
:101D500087DC9091720381E0911101C080E0F7016E
:101D6000818734C080917003813281F58091E800D1
:101D7000877F8093E80074DC8091720390917303F5
:101D8000882736E0969587953A95E1F7F70195878C
:101D900084871CC080917003813AC1F48091E8006F
:101DA000877F8093E8008091E80080FFFCCFF701F7
:101DB0008485958596958795969587958093F1006E
:101DC0008091E8008E778093E8004ADC0FB6F894A3
:101DD000BEBE0FBEADBE0F900F900F90DF91CF91A2
:101DE0001F910F91FF90EF90DF90CF90BF90AF9039
:101DF0009F908F907F906F900895FC01399627E017
:101E0000DF011D922A95E9F721E0FC01218724EFEB
:101E100031E03587248723E0248361E00196E4CB19
:101E20005F926F927F928F929F92AF92BF92CF926A
:101E3000DF92EF92FF920F931F93CF93DF9300D027
:101E40001F92CDB7DEB77C01ADB6BEB680916F03F1
:101E5000843009F08BC08091E4009091E500F70197
:101E6000228533852817390709F480C081818F7056
:101E70008093E9008091E80085FF78C08DB69EB61A
:101E8000408550E08DB79EB7841B950B0FB6F89434
:101E90009EBF0FBE8DBFEDB7FEB731966F011B829F
:101EA0001A82198260E070E0CF01A5D08E010F5F29
:101EB0001F4F960140E0BE016D5F7F4FC7010E943A
:101EC0009C01682EF70184859585892B41F021E0DE
:101ED00086859785892B09F020E0722E01C0712C30
:101EE000F701068117810115110589F049815A8191
:101EF000B801C6016AD055245394892B09F4512C9A
:101F0000F701408550E0B601C8016CD001C0512CEA
:101F100029813A81232BF1F0611004C0511002C0D5
:101F200070FE18C0F7018485958597878687818123
:101F30008F708093E9008B8181118093F10069811A
:101F40007A8140E050E0C601D7D98091E8008E77D1
:101F50008093E8008091E4009091E500F701938779
:101F600082870FB6F8949EBE0FBE8DBE0FB6F89452
:101F7000BEBE0FBEADBE0F900F900F90DF91CF9100
:101F80001F910F91FF90EF90DF90CF90BF90AF9097
:101F90009F908F907F906F905F90089500245527B9
:101FA00004C0080E591F880F991F009729F07695D5
:101FB0006795B8F37105B9F7802D952F0895EE0F49
:101FC000FF1F0590F491E02D0994FB01DC0104C092
:101FD0008D910190801921F441505040C8F7881B21
:101FE000990B0895FB01DC0102C001900D92415054
:101FF0005040D8F70895DC0101C06D934150504026
:10200000E0F70895DC01CB01FC01F999FECF06C091
:10201000F2BDE1BDF89A319600B40D9241505040A6
:10202000B8F70895F999FECF92BD81BDF89A992726
:1020300080B50895DC01A40FB51F4150504040F019
:10204000CB01840F951F2E9105D041505040D8F7F9
:102050000895262FF999FECF92BD81BDF89A019778
:1020600000B4021639F01FBA20BD0FB6F894FA9AE0
:0A207000F99A0FBE0895F894FFCF0F
:10207A000282190000015601190000000000000048
:10208A000183080000016F01080000000000000041
:10209A00008108000001770108000000000000002C
:1020AA004E020200182520BE58027A019A01260122
:1020BA003F0158010E03F201AA020E03F201AA021D
:0620CA00302E362E31001D
:00000001FF
